:020000040000FA
:1000000007309F0083169F011E308500F030860068
:1000100081138312EF30A40086000430A000A40CEA
:1000200024088600342006080F38A100A109031D0A
:100030001C28A00B0F280A28831600308600831284
:10004000A40924080F39A4002108F039A4042408C5
:1000500086001130A100A10321083C202402031DC9
:100060002B28210886003328FA30A300A200A20B17
:100070003728A30B362808008207113412341434B1
:100080001834213422342434283441344234443462
:1000900048348134823484348834303431343234D6
:1000A00033343434353436343734383438344134F6
:0A00B00042344334443445344634EE
:02400E00293F48
:00000001FF
